:03000000020030CB
:03000B00020119D6
:1000300011E020B0025132300021C200EA9002F1FA
:1000400093FBBB0A05115E02005BBB0B05118F021F
:10005000005B00A60308B878027870020037787059
:10006000760008B878FA787022E5301475F008A4A4
:10007000F53086F0E5305179510E080530B878F248
:10008000115EC201C20220B103D29622C29622782A
:10009000702001D57530017B00EB514986F0B5F039
:1000A000300B08B878F3115EE530B40107D203D203
:1000B0000231492274405149B40005B2B1B29622CE
:1000C000C28CD2B1C29631F1115ED296C2B1D28C3D
:1000D000220B08B878FB78700530BB40BC115E225B
:1000E000D2B0D2B7D290D291D292C295C294C293DA
:1000F000D296C2007A00C2B1C202C203C2017534F4
:1001000001115E758901C288C2A8D28CD2A975324C
:10011000257533FF5124D2AF22758A71758CB2C018
:10012000E0C0F031A0D53411200306753406020179
:1001300034753401300202B296200208D53605111A
:100140005E753699D0F0D0E0323000FDC200EA9002
:1001500002F193FBBB0B0302018EBB000302018E75
:10016000BB0A0302018EBB0930C2033000FBC20090
:10017000EA9002F193FBB40A0302018EB40B03026E
:10018000018E75F002A4C5F074405179510EC2027F
:1001900020B103D29622C29622D201C2038B302212
:1001A000D294D293C29531DE75F000701CD295C204
:1001B0009431DE75F0047011D294C29331DE75F083
:1001C00008D2937004E40201CB25F0B5020122CAE3
:1001D000700BD200753699C28C511ED28C227401DC
:1001E00030B70D043090090430910504309201E4D9
:1001F000227531FF7535FF74405149D531FD753198
:10020000FFD535F77531FF7535FFD5E0EE22753135
:10021000FF753515D531FD7531FFD535F7227532AE
:1002200025753315B2B3D532FD753225D533F5D2E8
:10023000B322753700E5379002FE93F5F0E53751AC
:10024000790537E537B441F222C0F0F5F051D440DA
:100250002574A04400C2E0519D4019E5F0519D4035
:100260001351D4401174A04400D2E0519D40055177
:10027000BFC3800251E8D0F02251D4401FC0E074C7
:10028000A04400C2E0519D400FD0E0C0E0519D402D
:1002900007E5F0519D4001C351E8D0E022C0F07560
:1002A000F0083392B500D2B400C2B4D5F0F4D2B5A0
:1002B0000000D2B400000000A2B5C2B4D0F022D237
:1002C000B5C0F075F008D2B400A2B533C2B4D5F011
:1002D000F5D0F022D2B5D2B430B50B30B408C2B5E7
:1002E00000C2B4C38001D322C2B500D2B400D2B5DB
:1002F00022FF0104070A020508000306090B010298
:1003000003040000000002020202000000000303D8
:1003100003030000000004040404000000000505BD
:10032000050500000000060606060000000007079D
:0F0330000707000000000808080800000000028E
:00000001FF
